:020000020000FC
:100000000DC0189518951895189518951895189568
:1000100090C01895189518951895A7C000E00EBFC8
:100020000FED0DBF00E808B901E007B906EC06B90D
:1000300003E00EBD0DEF0DBD0FE80CBD01E00CB9E6
:100040004FEE00EF0ABB0BBB07E007BB84E1DD27E7
:10005000C4E000E3402E502E602E702E789497FF5F
:1000600027C0EE24FF2430E1359A339A369A00C037
:100070003323E9F733983598F694E794F694E794A8
:1000800004EF11E030D01694079416940794E02CF6
:10009000F12C36D0A4E0BB27012D02951AD0012DFA
:1000A000906417D09F7B002D029513D0002D11D0A6
:1000B00000E205BF8895002705BFD1CF28E0C09892
:1000C000000F10F4C19A01C0C198C09A2A95B9F7DF
:1000D0000895E6E7F1E00F70E00FFB1F049196FD35
:1000E0000F7D0D930895222420E11695079510F4B5
:1000F0001E0C2F1C2794179407942A95B1F7089586
:1001000020E1222411240024FF27EE0CFF1C001CF8
:10011000111C221C2A9509F40895E3E002910D5F59
:1001200003FD00830081005D07FD0083E030B1F72F
:10013000ECCF0F930FB70F938A9511F484E1906879
:1001400000EF0BBBC2980991B9DFC29A042F007F60
:100150000BBB440F10F04FEEC4E00DEF0DBD0FE8E8
:100160000CBD0F910FBF0F91189504B1E00E05B1B2
:10017000F01E3A95189530F32AA2E1A424F220A0AB
:00000001FF
